:020000040000FA
:1000000006308A00732E0000831A0A28A500030E0A
:10001000A6000F288312A500030EA600A6140A0846
:10002000AD008A018313A50E0408A7002008A800CC
:100030002108A9002208AA002308AB002408AC006C
:1000400083128C308400001C27280C1895298B1EE5
:100050002B280B199D29270884002808A0002908AF
:10006000A1002A08A2002B08A3002C08A4002D0838
:100070008A00260E83008312250EA6188316090017
:100080000A108A100A11473E03188A0A82000034B7
:1000900000340034003480348034003400340034C0
:1000A000003400344034F034F034F034E034C03400
:1000B000803400348034C034E034E034E034E1345F
:1000C000C334C3348334033403340134013400347F
:1000D00081348F348F340F340034003400340034D2
:1000E0000034003400340034003400340034003470
:1000F00000348834F9340F340B3412349234A4347D
:10010000243449344B349234913420342E34213405
:100110009034903448344834243424341634FF3432
:10012000823455348834DD34003455348834DD3439
:10013000023414340034003400340034FE34FF340C
:100140001F34073400340034003400340034813468
:10015000FB34FB343334013400342034FF34FF34B7
:10016000F334F03470347034613421340134403469
:10017000F834FC344E346F347F343F341F3404344D
:1001800000340034003400340034003400340034CF
:10019000003400348034C0347E343334203420348E
:1001A00040344E349F34B23427344D347E347C3462
:1001B00000340134FF3401340034E63498347F34A1
:1001C000773400348034C0347F34553488345D341F
:1001D000203415340034003400340034003400344A
:1001E000003407340F340F340E340E340634073421
:1001F00007340634003401340F340734003400343B
:100200000034003403340F340F3404340034003429
:100210000034003400340034033407340E340E3418
:100220000F34073407340034003400340034003411
:100230000034003400340034003401340334023418
:100240000634043404340C340A34093419343C348C
:100250002D3467344234C2348434C434AB349834DB
:10026000C434443462342234333417340F34053404
:1002700002340134003400340034003400340034DB
:10028000003400340034003400340A148A100A1197
:1002900082077C3414341C34003400347834243421
:1002A0007834003400347C3440347C3400340034FE
:1002B000183444343034003400347C3454344434FE
:1002C00000340A148A100A11820701347D3415346F
:1002D0001D34013401347D34413401340134793426
:1002E00025347934013401341D3461341D34013432
:1002F00001345D340134FF3400340A148A100A11C9
:100300008207FF3401347D345534453401340134DF
:100310006D3411346D34013401347D3401340134D1
:1003200005347D340534013400340000FE308F0084
:100330006A308E000C108A112B2883160515831243
:10034000051DA9298316051583120519A229013057
:10035000B3068F0101308E000B118A112B288316F2
:100360000108C03906388100053083129000C03082
:100370008B0483160C14013083128F0095308E008D
:100380000730990083160508850003308312A0000A
:10039000A00BC82919088C11831699010C3085000F
:1003A00083129C2E08308316A800A8080319F1298F
:1003B000851283128512831627088039031DE529CB
:1003C000051283120512E8298316051283120516F9
:1003D000831685128312851603108316A70DA803B2
:1003E000D529831200348316051083120510831655
:1003F0002308A7008312D22100348316210807396D
:100400004038A200A3008312F321831620087F390D
:100410008038A200A3008312F32100348316051054
:100420008312051483162608A7008312D2210034F4
:100430008316051083120514831685108312851008
:100440006430F9007930840000080319352A01303E
:10045000A100A001A00B2A2AA10B292A4A30A00042
:10046000A00B302A332A800B272A8316851083128B
:10047000851421308316A3008312F321C83083161C
:10048000A3008312F32113308316A3008312F321F8
:1004900020308316A3008312F32109308316A300B2
:1004A0008312F3218316A001A1018312FD210130E3
:1004B000FA00F830F900F908031D612AFA08031957
:1004C0006A2A8316A60183120E2279080319FA03F9
:1004D000F9035B2A08308316A3008312F3210C3042
:1004E0008316A3008312F3218316A001A1018312B6
:1004F000FD219D2EFA01FB01FC01FA30FD007A0876
:100500008316A0007B08A1008312FD217C08FE0059
:100510007D087C077E0203189A2A7E0883169B00BA
:100520009C131C141A08FF007F08A60083120E22D9
:10053000FE0A882A8316A0010330A1008312FD2140
:10054000F9017908FC3C031CAE2A79084020FA0026
:100550008316A60083120E22F90AA12A00347C0811
:100560000739A0007D0CA2007C0CA100A20CA10CFC
:10057000A20CA10C1F30A2057F0821078400A10155
:10058000A10AA00AC42AA10DA00BC32AFE080319C0
:10059000CC2A21088004CF2AA10921088005003433
:1005A000FA01F9017A08013C031CE82A031DDC2A40
:1005B0007908943C031CE82A7A08FD007908FC00BD
:1005C000FE013C30FF00AF22F90A0319FA0AD22AD1
:1005D00000348316260807398312A0008316270CDF
:1005E0008312A2008316260C8312A100A20CA10C78
:1005F000A20CA10C1F30A205831628088312210724
:1006000084000008A100A00A062BA10CA00B052B5A
:1006100000348316A40124081A3C031C602B7E08B6
:10062000A500FF30A60083120E228316240822079D
:10063000A6002308A7000318A70A3C30A8008312CD
:10064000E922211C272B7F088316A5048312831619
:1006500024082207A6002308A7000318A70A1B30B6
:10066000A6070318A70A3C30A8008312E922211C20
:100670003D2B83162008A504831283162408220725
:10068000A6002308A7000318A70A3630A6070318F8
:10069000A70A3C30A8008312E922211C532B8316A1
:1006A0002108A504831283162508A60083120E22B2
:1006B00083162508A60083120E228316A40A0B2B8C
:1006C000FF30A60083120E22003483168515831294
:1006D0008519902B831605158312051D8F2B831604
:1006E0000515831205196F2B0F08A3000E08A00033
:1006F0000F082302031D742B2008FF3CFA00FF3073
:10070000FB002308031C230FFB027B08FD007A0873
:10071000FC000130FE003C30FF00AF220024652BBE
:100720008B160130810000341F308316A000023088
:10073000A1008312FD21F9017908173C031CA92BA4
:1007400079084521FA008316A60083120E22F90AC1
:100750009C2B8316A0010530A1008312FD21F90115
:100760007908173C031CBD2B79086121FA00831618
:10077000A60083120E22F90AB02B41308316A00086
:100780000530A1008312FD21F9017908123C031CF8
:10079000D22B79087D21FA008316A60083120E223F
:1007A000F90AC52BAC2E79080739A000790CA100F5
:1007B000A10CA10C1F30A10521087B078400A10119
:1007C000A10AA00AE42BA10DA00BE32BFA08031940
:1007D000EC2B21088004EF2BA109210880050034AF
:100800008316A001A1018312FD21FD017D081A3C80
:10081000031C362CFC308316A60083120E222430D3
:10082000FC008316A7017D08A6003C30A8008312B7
:10083000E922211C1D2C1830FC041B307D07831677
:10084000A701A6003C30A8008312E922211C2A2C13
:10085000C030FC047C088316A60083120E227C089C
:100860008316A60083120E22FD0A062CFC30831686
:10087000A60083120E228316A0010130A10083126C
:10088000FD214930FE000630FF0030308316A00005
:100890008030A100A3013630A20083120923831601
:1008A000A0010230A1008312FD219230FE00013030
:1008B000FF000C308316A0006030A100A3016C3053
:1008C000A200831209238316A0010330A100831222
:1008D000FD212430FE000330FF0018308316A000F5
:1008E000C030A100A301BD30A200831209238316EA
:1008F000A0010430A1008312FD214930FE00063022
:10090000FF0030308316A0008030A1000130A3002A
:100910000E30A200831209238316A0010530A10026
:100920008312FD219230FE000130FF000C3083164F
:10093000A0006030A1000130A3004430A200831267
:1009400009230034A101A201A001A30183162308F9
:10095000031DAD2C22080319D12C1030A400031064
:10096000A00DA10D8312A00DA30D831623088312E1
:100970002302031DBF2C8316220883122002031CAE
:10098000CC2C831622088312A002031CA303831617
:1009900023088312A3020314A10DA20D8316A40B36
:1009A000AF2C83120034FF017C088316A1007B0862
:1009B000A000A3011B30A2008312A2242008FD0086
:1009C0007C088316A1007B08A000A3011B30A200B5
:1009D0008312A2242108FE00FD08031DF12C003023
:1009E000F22C01308316A000FE08031DF92C003004
:1009F000FA2C0130A0051B307B02A1007C08A2006C
:100A00000030031C0130A2020130A1020030031C9F
:100A10000130A2022208A7002108A6003C30A8004D
:100A20008312E9220030211801300139013C0319F9
:100A30001B2D00301C2D0130831620050319222D9B
:100A40000130FF07FE08031D272D0030282D01303F
:100A5000A0001B307B02A1007C08A2000030031C18
:100A60000130A2022208A7002108A6003C30A800FD
:100A70008312E9220030211801300139013C0319A9
:100A8000432D0030442D01308316200503194A2DD3
:100A90000130FF077D08193C0318502D0030512DFF
:100AA0000130A000FE08031D572D0030582D0130E5
:100AB000A0051B307B02A1007C08A2000030031CB3
:100AC0000130A2020130A1070318A20A2208A700E0
:100AD0002108A6003C30A8008312E922003021182A
:100AE00001300139013C0319772D0030782D013098
:100AF0008316200503197E2D0130FF07FD08031D15
:100B0000832D0030842D0130A00001307B02A10034
:100B10007C08A2000030031C0130A2022208A700BA
:100B20002108A6003C30A8008312E92200302118D9
:100B300001300139013C03199F2D0030A02D0130F7
:100B4000831620050319A62D0130FF077D08193CE7
:100B50000318AC2D0030AD2D0130A00001307B0713
:100B6000A1007C08A2000318A20A2208A7002108FD
:100B7000A6003C30A8008312E92200302118013081
:100B80000139013C0319C62D0030C72D01308316F1
:100B900020050319CD2D0130FF07FD08031DD22DBF
:100BA0000030D32D0130A0007E080D3C0318DA2D53
:100BB0000030DB2D0130A0051B307B07A1007C0835
:100BC000A2000318A20A0130A1020030031C013068
:100BD000A2022208A7002108A6003C30A800831228
:100BE000E9220030211801300139013C0319FA2DA6
:100BF0000030FB2D0130831620050319012E013032
:100C0000FF077E080D3C0318072E0030082E013028
:100C1000A0001B307B07A1007C08A2000318A20AD9
:100C20002208A7002108A6003C30A8008312E92270
:100C30000030211801300139013C0319212E003008
:100C4000222E0130831620050319282E0130FF07BC
:100C50007D08193C03182E2E00302F2E0130A000E5
:100C60007E080D3C0318362E0030372E0130A005CB
:100C70001B307B07A1007C08A2000318A20A0130E8
:100C8000A1070318A20A2208A7002108A6003C30E9
:100C9000A8008312E9220030211801300139013CFB
:100CA0000319542E0030552E0130831620050319E8
:100CB0005B2E0130FF077F088312A1000034790802
:100CC0000739A000790CA100A10CA10C1F30A105CF
:100CD00021087A0784000008A100A00A702EA10C48
:100CE000A00B6F2E003403081F3983005F30A00073
:100CF0002130840083138001840AA00B7B2E2030D6
:100D0000A000A030840083138001840AA00B842EED
:100D1000A00184011F308305613083168F000F0806
:100D200083121F1383161F109F101F119F1107306E
:100D3000831299003314AF29182A7A22D022013065
:100D4000F900652383160C1083120024F6011B3072
:100D5000F5003318C62E942B3318C62E831685152E
:100D60008312851DC52E8316851583128519B32E12
:100D700033148B1283160C1483127A22D022013082
:100D8000F900652383160C108312AC2EF001700855
:100D90001A3C031C062FFC017008FB00D324210819
:100DA000F4007008F900FA013430FB00D323740812
:100DB000033C0319DD2E0030DE2E0130F9007408EB
:100DC000023C0319E52E0030E62E0130FA008316AE
:100DD000A7017008A6003C30A8008312E922003069
:100DE000211801300139013C0319F82E0030F92E89
:100DF00001307A0579040319042F7008F9000130D5
:100E0000FA003430FB00D323F00AC72EEF016F083D
:100E10000D3C031C9B2FF00170081A3C031C5B2F38
:100E200070087507F9007608FA000318FA0A7A08BC
:100E3000FC007908FB00D3242108F4007008F900B5
:100E4000FA013830FB00D3237408033C03192A2F1E
:100E500000302B2F0130F9007408023C0319322FA7
:100E60000030332F0130FA0070087507FB00760858
:100E7000FC000318FC0A7C088316A7007B08A60068
:100E80003C30A8008312E9220030211801300139DA
:100E9000013C03194D2F00304E2F01307A057904A3
:100EA0000319592F7008F9000130FA003830FB009F
:100EB000D323F00A0C2FF10171081A3C031C812F77
:100EC0001B307502F9007608FA000030031C01306F
:100ED000FA0271087907F7007A08F8000318F80A8F
:100EE0007108F9003430FA005F267808FD007708B1
:100EF000FC00FE012118FE0A3C30FF00AF22F10A7F
:100F00005C2FF20172081A3C031C952F7208F9003D
:100F10003830FA005F267208F900FA012118FA0A3F
:100F20003430FB00D323F20A822F1B30F50703185D
:100F3000F60AEF0A072FF30173081A3C031CC12FAE
:100F40001B307502F9007608FA000030031C0130EE
:100F5000FA0273087907F7007A08F8000318F80A0C
:100F60007308F9003430FA005F267808FD0077082E
:100F7000FC00FE012118FE0A3C30FF00AF22F30AFC
:060F80009C2FA52E63006A
:0207FE00803445
:10420000C000700098000C000600020003000100CE
:1042100001000300C200A6006C009800F0004000FE
:10422000E0001000A8004000E8001000A00000001E
:10423000000000000000C000E000F00038001C009A
:104240001C00CE00EE00EE00FE00E800E0004000A2
:10425000000000008000800080008000C000E000BE
:10426000F000F000000000000000C000E00070005E
:104270007000F000E000C000C000C000C00080007E
:104280000000000000000000C000E00070007800A6
:10429000FC00FC00FC00200000000000000000000A
:1042A0000000000000000000FF005400A9005100C1
:1042B0005300AA002A000600060006001E00E200C5
:1042C0000900AA00FF0054008A0051002A000400DF
:1042D00002000100000000000000000002000700D2
:1042E0000F001C001C00380038003F003F003F005A
:1042F000010000000000000008003E003F007100C7
:104300007100710071007F007F003F0000002000FD
:10431000FF003F00070000000000000007003F0012
:104320007F0023000100010003007E007C003200BA
:104330001F003F00720073007B003900380000004E
:10434000000000000000000000000000000000006D
:104350001F0035006A00D500CB008000800080007F
:104360008000800080008000C700780027003D00AA
:104370000A00000000000000000000000000000033
:10438000F000F800FC00FC001C008C00CC00FC00DD
:10439000F800F000E000FE00FF00C700E300E300CB
:1043A000C7004600060000000000000000000000FA
:1043B0000000000000000000C00060003000180095
:1043C0000C00E400AE002A0053005100A1002300BD
:1043D0004200860044002C002800180030006000D5
:1043E000C000C000000040008000C000200040006D
:1043F0008000C000800000000000000000000000FD
:02400E00D430AC
:00000001FF
